:1000000003C4000039C4000037C4000035C4000038
:1000100033C4000031C400002FC400002DC4000010
:100020002BC4000029C400000C94932F0C947B3047
:100030000C94482F21C400001FC400001DC4000000
:100040001BC4000019C4000017C4000015C4000040
:1000500013C400000C946F2F0FC400000DC40000E7
:100060000BC4000009C4000007C4000005C4000060
:1000700003C4000001C40000FFC30000FDC3000072
:10008000FBC30000F9C30000F7C30000F5C3000084
:10009000F3C30000F1C30000EFC30000EDC3000094
:1000A000EBC30000E9C30000E7C30000050109023B
:1000B000A10185020901A1000509190129081500FE
:1000C0002501950875018102050109300931158165
:1000D000257F95027508810609381581257F9501D0
:1000E00075088106050C0A38021581257F95017572
:1000F000088106C0C005010980A101850319012AF4
:10010000B700150126B700950175108100C0050CD8
:100110000901A101850419012AA002150126A002E6
:10012000950175108100C005010906A1018506052C
:100130000719E029E71500250195087501810205D9
:1001400007190029EF1500250195F07501810205B9
:10015000081901290595057501910295017503910D
:1001600001C00660FF0961A1010962150026FF00B8
:100170009520750881020963150026FF00952075FA
:10018000089102C005010906A101050719E029E748
:1001900015002501950875018102950175088101F9
:1001A0000507190029FF150026FF0095067508812F
:1001B000000508190129051500250195057501910E
:1001C00002950175039101C00000000000000000CD
:1001D000000000000000000000000000000000001F
:1001E0000000000000000000000000007E0F00D4AE
:1001F000FFFFFFC7000000780000000000000000C3
:100200002A2B280000000000000000000000000071
:1002100000000029000000002C1E3420212224347C
:100220002627252E362D3738271E1F20212223244E
:1002300025263333362E37381F0405060708090AEA
:100240000B0C0D0E0F101112131415161718191A86
:100250001B1C1D2F3130232D350405060708090A04
:100260000B0C0D0E0F101112131415161718191A66
:100270001B1C1D2F3130354C09025B00030100A00F
:10028000FA09040000010301010009211101000124
:10029000224400070581030800010904010002034C
:1002A000000000092111010001222200070582033C
:1002B00020000107050303200001090402000103D7
:1002C00000000009211101000122B6000705840386
:1002D00020000112010002000000084C5A5349108E
:1002E00000010203011C037600690061006C003A02
:1002F00000660036003400630032006200330063A1
:100300000000000E0349005200490053003600353A
:100310000000000A037A006C006B00620000000419
:1003200003090429001E001F0020002100220023D1
:100330000024002500260027002D002E0031002A71
:10034000004C002B0014001A000800150017001CB8
:100350000018000C00120013002F0030003100A91B
:10036000000000215204001600070009000A000BDB
:10037000000D000E000F003300340031002800AAE9
:10038000000000E10031001D001B000600190005FF
:100390000011001000360037003800E5005200AEB2
:1003A000000000E000E300E2002C0000000000007C
:1003B00000000000000000E600E400500051004F83
:1003C00000000035003A003B003C003D003E003F8D
:1003D0000040004100420043004400450001004C41
:1003E000004C0001000100010001000100010001BA
:1003F00000AC00AE00AB00010001000100010001F3
:100400000000000100010001000100010001005096
:1004100000510052004F00010001000100010001E5
:1004200000000001000100010001000100010001C5
:10043000000100010001000100010001004B00016A
:1004400000000001000100010001000000000000A8
:1004500000000000000000010001004A004E004DB5
:1004600000000001000100A70341169516000002DC
:10047000000200A30341169516000003000100A826
:1004800003411695160000040002008D03411695E5
:10049000163F0805000100A9034116951600000645
:1004A0000002008F0341169516000007000200A508
:1004B00003411695160000090002009103411695AC
:1004C0001648080A00020093034116951648080BC7
:1004D00000020095034116951648080C000200978B
:1004E000034116951648080D000200990341169520
:1004F0001648080E0002009B034116951648080F87
:100500000002009D03411695164808100002009F46
:100510000341169516480811000200A103411695E3
:1005200016480812000200AB03411695160000138E
:10053000000200AD0341169516000014000100AF43
:10054000034116951600001500000000006D08A577
:1005500010000016000100AA035816AC1600001780
:10056000000101AA035816AC16000018000102AAE7
:10057000035816AC16000019000200B1034116958D
:100580001600001A000103AA035816AC1600001B3F
:10059000000200B303411695160000FD377A585A41
:1005A000000004E6D6B446020021011600000074E3
:1005B0002FE5A3E004D101A95D003D8889C654362A
:1005C000C3174FE4E0DC0B8B21188F1A823BA08607
:1005D000C083B00797309A48E3293EDAA586F30B2B
:1005E000C2FF4D9C99E6001862DB9AD3A3CCBDA54F
:1005F000890E73A82273DF0D0EC1E4F667C142991C
:100600005B2D1E01B2003D6B1AA002DF364F0AC2FD
:1006100056C7A463606EB92C7E96A4483C65E3512E
:1006200031D717B701A356C7283F724EE3AB0FCCA3
:10063000FD507C9BBB1018C983E974D37393E7F01A
:100640005DCA8BF1F607A308F117828CAE0C7C30E3
:10065000BCE768A929D895443E18F0DEEA96EBF984
:10066000DB674BA11B23622827F335105FF8A50039
:10067000A4F30AD671362517CEA62412438BDCC20A
:10068000FB4618436A2675E00D3706C636FB289EE2
:10069000B5D4D9C9657CB469D78EFD74EF8B6DE88C
:1006A000CD5F1EAF6C3691AEA6533F96FC1B910BEF
:1006B000E0240DF6A87EE013693A5E134B46730101
:1006C000A2F6FDB60C9F15D1605FFB7AE1A7B27070
:1006D000ABC7B09014FC3335E1DA06C0A4041DE0CA
:1006E0009E80ADCD011DB5327094EECFD2A485426F
:1006F000A892931F01E45ECB75263A9ED5C8E01FF1
:10070000029F4DE75AAB3C5BE05935EA3DC8CBADA3
:10071000DF46F3B41230A389EA2010F4D6A933AE31
:10072000DD889B1B94312E341A2D521DAC7CE57A4A
:10073000403D9544D44AA3358F8A7C1EDAA1254BCF
:1007400019AF994A2534D0E96746550B53B79568D8
:10075000C4BB6BF0595C49D6BBEF22579C8EC8884E
:10076000B893000000000052D85497D537CA6000F3
:1007700001C503D2090000976B5C46B1C467FB0258
:100780000000000004595A4C4C4C4C4C4C525252F4
:10079000525252520052524C4C4C4C4C4C525252AF
:1007A000525252525252004C4C4C4C4C4C5252529F
:1007B000525252005252004C004C4C4C4C4C525233
:1007C000525252525252004C4C4C2A00000000002F
:1007D00000525252525200504F52514A4D4B4E2AE3
:1007E0004C2F30B6B7ABACBBBCA9AABDBECFD0CDE9
:1007F000CEDBDCD9DA0D0E0B0F1A0508050905074B
:100800001811130408120C0011241FBECFEFDAE0F8
:10081000DEBFCDBF04B603FE18C08091BA0390912D
:10082000BB03A091BC03B091BD038730904BA740A0
:10083000B04B59F41092BA031092BB031092BC0350
:100840001092BD03E0E0F8E3099511E0A0E0B1E00B
:10085000EAE7F4E602C005900D92A63BB107D9F78E
:1008600023E0A6EBB1E001C01D92AA3BB207E1F77D
:100870000E94B4280C94C831C3CB9C01FB019A950B
:1008800081159F4120F5832F8170B32FB270AA2765
:10089000732F74706627532F5870442734FF0DC090
:1008A0008295807FAB2B09F08062672B09F0806412
:1008B000452B09F0806809950895AB2B09F08260FB
:1008C000672B09F08460452BB1F38860F4CF80E09A
:1008D000F2CF0C94F3300895982F92959F7024E0F6
:1008E000911102C020E0982F892F86958695811559
:1008F00011F02E5F982F892F8695820F0895282F4B
:1009000092959F70963099F060F4925F9F7092304C
:1009100030F4203FB1F038F481E0283E38F080E038
:1009200008959A5FF3CF81E0243FC9F7089591E0DD
:10093000813F09F090E081E0283E08F080E0892BBB
:10094000089581E0089580932F03089580933003E4
:10095000089521E030E001C0220F8A95EAF78091E6
:100960003003822BF3CF21E030E0A90102C0440F15
:10097000551F8A95E2F7CA0180959091300389232B
:10098000E5CF953080F5803170F540E1949F90017E
:100990001124280F311D877041E001C0440F8A9552
:1009A000EAF783E0369527958A95E1F7F901EE0F8E
:1009B000FF1FE20FF31FE257FD4F80E090E070E071
:1009C0005191DF019B01082E02C0369527950A94AC
:1009D000E2F7217021952527242325272E930196C0
:1009E0008330910569F70895953078F5803168F581
:1009F00040E1949F90011124280F311D982F97708A
:100A000083E0369527958A95E1F7F901EE0FFF1FF0
:100A1000E20FF31FE257FD4F40E050E080E02191EC
:100A200030E0092E02C0369527950A94E2F721702E
:100A30003327042E01C0220F0A94EAF7822B4F5F5E
:100A40005F4F4330510559F7089580E00895909124
:100A5000300321E030E0F90101C0EE0F8A95EAF79A
:100A6000D90102C0AA0FBB1F6A95E2F7EA2B01C0A9
:100A7000220F4A95EAF7892F8E23E81303C0892FA6
:100A8000822B64CF2095822F8923FBCF80918D020A
:100A900090E020E0022E001C0008281709060CF048
:100AA00008952F5FF7CFCF93DF93EC01DB018C81AB
:100AB000813059F514968C911497813031F5E98184
:100AC00080E1E89FF00111248881E80FF11DE957CA
:100AD000F84F94919A32C9F01196EC91119780E1F8
:100AE000E89FF00111248C91E80FF11DE957F84FB0
:100AF000E49181E09E1301C080E091E0EA3209F0C8
:100B000090E0892BDF91CF91089581E0FBCF9C018C
:100B1000809131038D79811119C0211540E5340789
:100B200080F4211580E23807C0F42333310511F138
:100B3000D0F481E02E31310590F42430310530F0CD
:100B40000895C90196558115914010F080E00895EF
:100B5000C901805F96450797C8F33327E6CF2C324B
:100B60003105A1F708952653310981E0233031057D
:100B700038F3ECCF81E0089580913B0390913A03E4
:100B8000981301C008958F5F8770FACF9091350355
:100B90008095892380933503282F2770211110C059
:100BA000891771F09091B60392FF0AC086958695D9
:100BB0008695D9DE109235031092370310923603D2
:100BC000089590913103982B909331030895982FB5
:100BD000909580913103892380933103089580910A
:100BE0002D03811531F010922D0310922C031092D9
:100BF0002B030895803E9105D9F1C8F48133910506
:100C000009F482C048F48932910509F472C08A322D
:100C1000910509F480C0089589339105E9F082387F
:100C20009105D1F08533910509F45EC00895843EA5
:100C30009105D9F148F4823E910539F1833E910541
:100C400049F181EE90E00895863E9105C9F1873E15
:100C5000910509F43EC008952091B5032370211138
:100C600064C02091B60323FF14C089E290E0089588
:100C70002091B50320FD45C03091B60330FF09C077
:100C800024FD24C083EE90E008952091B50322FD59
:100C9000F7CF08952091B50322FD44C03091B603EB
:100CA00030FD43C024FFF5CF11C02091B60321FFD2
:100CB000F0CF8091B50384FD09C087EE90E00895E0
:100CC0002091B50323FFE5CF24FFF7CF80E090E02C
:100CD00008952091B50323FD2BC03091B60331FF59
:100CE000E1CF84EE90E008952091B50325FFD1CFA8
:100CF000BCCF2091B50325FD1EC02091B60323FF74
:100D0000C8CF89E390E008952091B50326FFC1CFB5
:100D10008AE290E008952091B50326FFBACF81E3DF
:100D200090E0089582EE90E0089580EE90E00895BE
:100D300086EE90E0089585E390E008959091B503E4
:100D400092FF10C041E0282F2471243009F040E0C8
:100D500031E0282F2871283009F030E0431711F0D6
:100D60002CE0822793FF10C041E0282F247124310A
:100D700009F040E031E0282F2871283109F030E0F7
:100D8000431711F02CE082273091B60330FF10C0DA
:100D900051E0282F2171213009F050E041E0282F47
:100DA0002871283009F040E0541711F029E082271B
:100DB00031FF10C041E0282F2171213109F040E0BE
:100DC00031E0282F2871283109F030E0431711F065
:100DD00029E0822794FD877E08951F93CF93DF93A8
:100DE00009DFEC01811522E5920708F052C0811558
:100DF00040E5940708F0CDC0803E910520F58D3C7C
:100E0000910508F0A1C0883A910570F4853A9105E2
:100E100008F097C081309105B9F10497813A9105A6
:100E200098F1C0E0D0E030C0885A91094B97C8F7DC
:100E3000C85AD0E0CC0FDD1FC75BDE4F0990D881C8
:100E4000C02DD46421C0811550E49507B0F4C115BC
:100E500080E2D80708F0B3C0C83ED105A8F0CE01A3
:100E60009A9581159F41E8F68D2F68DF182FCE01E6
:100E70009927C0DEEC01D12B07C09927BBDECC2718
:100E8000DF70C82BD92BD06ACE01DF91CF911F9193
:100E90000895803842E59407C8F5803652E59507F5
:100EA00008F05BC0C03482E5D807D0F4C03292E5C8
:100EB000D90708F04BC08C2F8695869520E2829F3B
:100EC000C0011124C37021E030E0A90102C0440F29
:100ED000551FCA95E2F7EA01C82BD92BDD68D4CF9C
:100EE0008C2F86958695877050E2859FC0011124CE
:100EF000C37021E030E0A90102C0440F551FCA951C
:100F0000E2F7EA01C82BD92BDC68BECF803C52E562
:100F1000950758F48F71C03AD245A0F590E0982F0C
:100F20008827EC01C46FD06AAFCF805C9245809770
:100F300008F077CFDC2FCC27CC27DF71C06FD06AC9
:100F4000A3CFA497D064A0CFD0659ECFCF71D0E0BF
:100F5000DC2FCC27C16FD06A97CF86958695877096
:100F600020E2829FC0011124C37021E030E0A9017A
:100F700002C0440F551FCA95E2F7EA01C82BD92BCE
:100F8000DA6882CFDBDEC82FD0E0DC2FCC27D0623E
:100F90007BCF8F71D3DE93E0CC0FDD1F9A95E1F705
:100FA000CC27DF70282F30E084FF05C050E1859FFB
:100FB000900111243327C22BD32BD06965CF8D2FFD
:100FC0008F71BCDE182FCE01992714DEEC01D12BD6
:100FD000DECF80E00895F894E82FE295EF70F0E01E
:100FE00041A18F7021E030E0B90102C0660F771F88
:100FF0008A95E2F7CB01962F9095942391A392A125
:10100000892B82A378940895FB01811520E2920731
:1010100028F4811541E0940738F408959C0130527A
:101020002115304348F00895392F94FF02C03295BE
:10103000307F2081232B208399270895462B22FF80
:101040000FC0982F92959F708F70892B962F929535
:101050009F706F70692B942F92959F704F70492BE2
:10106000982F9623961309C050E04095509590E034
:101070004823592381E0452B09F080E008958091B1
:101080008D0390918E039093110180931001089528
:10109000EDE8F3E0848195812AE030E0B9010E9417
:1010A000C6306093140186818093150182858093F8
:1010B000030184858093020186859785B9010E948A
:1010C000C6306093120180898093130182898093D6
:1010D00001018489809300010895EF92FF920F939C
:1010E0001F93CF93DF93FB018FEF9FEF44305105A8
:1010F00008F45FC04091B50341FB882780F990E078
:10110000880F991F42FB002700F910E0000F111F04
:10111000000F111F802B912B40FBEE24E0F8F12CE7
:101120008E299F2943FB222720F9C22F50E0D52F7B
:1011300053E0CC0FDD1F5A95E1F78C2B9D2B44FB20
:10114000222720F950E1259F90011124822B932B17
:1011500045FB222720F950E2259F90011124822B84
:10116000932B46FB222720F950E4259F9001112460
:10117000822B932B47FB222720F940E8249F9001E4
:101180001124822B932B2091B603322F3170932B95
:1011900026952170B22FBB0FA0E08A2B9B2B092E26
:1011A000000CAA0BBB0B80839183A283B38380E0E6
:1011B00090E0CDB7DEB7E6E00C943231AC0123E02D
:1011C000969587952A95E1F78E719927FC01E05055
:1011D000FE4F0190F081E02D4F70552721E030E067
:1011E00002C0220F331F4A95E2F7611541F0E22B4E
:1011F000F32B80509E4FDC01ED93FC9308952095D6
:101200003095E223F323F5CF0F931F93CF9301E0A3
:1012100010E0082E01C0000F0A94EAF7C0912A03DB
:101220009C2F9023911115C090913503969596951A
:101230009695891306C010923503109237031092C9
:10124000360387DBC027C0932A03CF911F910F91EC
:10125000089589DBF7CF282F35EB2303C001112434
:1012600097FF04C080589109892F089580589F4F97
:10127000FBCF8091AE02609195037091960380FF41
:1012800014C020910301269FC001279F900D1124B7
:10129000BC01769567957695679560387105F0F590
:1012A00061157105E9F1862F089581FF0BC020912A
:1012B0000301269FC001279F900D1124BC01769544
:1012C0006795EBCF82FF09C0809103019B01829F4C
:1012D000B001839F700D1124E0CF8091AD02811584
:1012E000E1F29091020120910301891738F0CB01BE
:1012F000289FB001299F700D1124CFCF289F900106
:101300001124269FA001279F500D369F500D1124B8
:10131000692F70E0CA010E94C630BFCF8FE70895E1
:1013200081E008958091AE0280FF0CC060910101C0
:1013300070E075956795759567956115710549F12B
:10134000862F089581FF06C06091010170E07595B8
:101350006795F3CF6091010182FD0BC09091AC02C3
:101360009115A1F06091000180910101961738F06C
:10137000682F70E06038710500F38FE70895899F4A
:10138000C001112470E00E94DA30F4CF61E070E017
:10139000D7CF81E0089590910C0389029001112428
:1013A00037FF03C080930C0308952F3731051CF4D9
:1013B000980F90930C0308959C0180E090E0F90150
:1013C000E80FF91FE491E41307C091E08927F901C0
:1013D000E80FF11D849108950196861780F380E04F
:1013E0000895E0917302F0917402309739F0019002
:1013F000F081E02D309711F00995089580E008956F
:10140000A3E0B0E0E6E0FAE00C941A319C01809190
:10141000FE019091FF0182179307B1F03093FF0115
:101420002093FE01E0917302F0917402309761F015
:101430000084F185E02D309739F083E089833B8388
:101440002A83CE01019609952396E2E00C94363169
:10145000A3E0B0E0EEE2FAE00C941A319C01809136
:10146000FC019091FD0182179307B1F03093FD01CB
:101470002093FC01E0917302F0917402309761F0C7
:101480000084F185E02D309739F084E089833B8337
:101490002A83CE01019609952396E2E00C94363119
:1014A00090911801913091F0AAEBB1E0EFEF90E04C
:1014B0002D91821751F0EF3F19F4211101C0E92F4E
:1014C0009F5F9630A9F7EF3FC9F408959091B50357
:1014D00097FFEACFE82FE695E695E695803FA8F7D7
:1014E000F0E0E054FE4F877021E030E001C0220FB1
:1014F0008A95EAF78281822B828308950E2E000C52
:10150000FF0BE854FE4FF8CF90911801913021F471
:101510009091B50397FD0CC0EAEBF1E0919189132E
:1015200002C0DF011E9251E0E03CF507B9F70895D3
:10153000E82FE695E695E695803FC8F7F0E0E054A1
:10154000FE4F877021E030E0A90102C0440F551F13
:101550008A95E2F7CA018095928189238283089552
:101560008091170108952FB7F8948091F801909118
:10157000F901A091FA01B091FB012FBF089580916C
:101580008F0390919003892B89F0EDDF20912B033D
:1015900030912C03AC01421B530B9A0181E0409126
:1015A0008F03509190032417350708F480E00895C5
:1015B000CF93DF93C091310380913403C82B809186
:1015C0002D038115E1F080918F0390919003892B79
:1015D00019F0D5DF811103DBD0912D038091180123
:1015E000813021F48091B50387FD0DC086E02AEBA0
:1015F00031E090E0815058F49111F1DACD2B8C2F2D
:10160000DF91CF9108958EE122EC31E0F2CFF90124
:1016100041919F01411571F39F5FECCF962F20916F
:10162000B60322FF0EC0682F660F660F660F692B88
:10163000609335038ED997DF9093370380933603F9
:10164000089587C990912D03292F2823211559F03A
:101650008095892380932D03811531F084DF809359
:101660002B0390932C03089580E090E0F8CFCF9364
:10167000C82F8091B60382FF0BC080912D038C1779
:1016800039F071DF90932C0380932B03C0932D03CB
:10169000CF91089568DF2091B1023091B202232BDF
:1016A000211521F08093390290933A022091B302E0
:1016B0003091B402232B211521F0809337029093AF
:1016C0003802E0917302F0917402309759F006806D
:1016D000F781E02D309731F082E08093AF028FEAFE
:1016E00092E009950895611509F441C0E3E3E80F1C
:1016F000E33148F4F0E0E653FE4C0C94ED30B9DDF4
:1017000081958093B202C6CFB4DDFBCFB2DD819567
:101710008093B102F8CFADDDFBCF04DE8093B3023E
:10172000F2CF00DE8195FACFFDDD81958093B40282
:10173000EACFF8DDFBCF815D990B21E030E001C0FD
:10174000220F8A95EAF78091B002822B8093B00233
:10175000DACF8091AE0281608093AE02D4CF8091C7
:10176000AE028260F9CF8091AE028460F5CF4091E5
:10177000B1028D3C59F48091B20287FF0DC01092E6
:10178000B202411559F41092AD0208C08E3C81F4AA
:101790008091B20218169CF3411581F08091B3023A
:1017A0009091B402892B8111AECF1092AC02ABCFD5
:1017B0008F3C41F447FFF0CF1092B1028091B2020A
:1017C0008115E0CF803D19F41416B4F3E5CF909164
:1017D000B302893D29F41916FCF61092B302DCCF4E
:1017E0008A3D19F497FFD8CFF8CF9091B4028B3D82
:1017F00029F497FFD1CF1092B402CECF8C3D19F4CB
:101800001916CCF3C9CF9FE2980F983090F4815D00
:10181000990B21E030E0B90102C0660F771F8A956D
:10182000E2F7CB0180959091B00289238093B002BA
:10183000B3CF8D3D31F48091AE028E7F8093AE02A6
:10184000ABCF8E3D21F48091AE028D7FF7CF8F3DDF
:1018500009F0A2CF8091AE028B7FF0CF2FB7F89422
:101860006091F8017091F9018091FA019091FB016A
:101870002FBF0895FC019B018091EE019091EF0133
:101880008617970740F0672B29F48091E8008E7740
:101890008093E800C90140E0009741F4411106C07F
:1018A0008091E80082FF2FC080E0089520914C02D3
:1018B0002115A9F12530A9F12091E80023FD2DC0C3
:1018C0002091E80022FDECCF2091E80020FFE4CF3A
:1018D0003091F3002091F200009719F02830310583
:1018E00058F041E02830310509F040E02091E8004F
:1018F0002E772093E800D0CF41914093F1000197DB
:101900002F5F3F4FE9CF80914C02811541F0853028
:1019100041F08091E80083FFC3CF81E0089582E029
:10192000089583E008958091E80187FF13C08091B6
:10193000E80082FF06C08091E8008B778093E80082
:10194000089580914C028111F2CF089580914C024C
:101950008115D9F38091E80080FFF8CF8091E800ED
:101960008E77ECCF2091E4003091E50095E6A90157
:101970002091EC00822F817020FF06C08091E8004A
:1019800080FF06C080E008952091E80022FD1AC083
:1019900080914C02811589F0853089F08091EB00AF
:1019A00085FD0FC02091E4003091E50042175307F8
:1019B000F9F29A95E1F684E0089582E0089583E0D3
:1019C000089581E00895E8EDF0E080818E7F8083C6
:1019D0001092E2001092DA001092E100A0EEB0E066
:1019E0008C9181608C9380818F77808319BCA7ED67
:1019F000B0E08C918E7F8C9380818F7E808310925B
:101A0000E7010895E0917302F0917402309739F084
:101A10000284F385E02D309711F060E20995089576
:101A2000982F9093E900891771F07091EC00209144
:101A3000ED005091F00021FD09C09F5F973089F7BC
:101A40008093E9000895762F242F50E03091EB0029
:101A50003E7F3093EB003091ED003D7F3093ED0001
:101A60003091EB0031603093EB007093EC002093E9
:101A7000ED005093F0002091EE0027FDDECF089599
:101A8000A0E0B0E0E6E4FDE00C941431C8EDD0E055
:101A900088818F7E8883E7EDF0E08081816080839C
:101AA00084E082BF81E08093E70188818E7F888314
:101AB00002EE10E0F80110821092DA0081EEC82EDA
:101AC000D12CF601108288818F7788838881806885
:101AD000888388818F7D888319BC10924C02109274
:101AE000E60110922B021092E50190EEE92EF12C06
:101AF000F70180818B7F808388818160888342E0C9
:101B000060E080E08DDFF60180818E7F8083F801C8
:101B1000808181608083808188608083F7018081FB
:101B20008E7F8083888180618883CDB7DEB7E8E0CF
:101B30000C943031E0913B0390913A0329E0E91392
:101B400002C080E00895AE2FB0E02E9FF001112476
:101B5000E45CFC4F3181361306C03081381303C07A
:101B60003581341304C0FD013196E770E8CF81E080
:101B700008959C012115310509F408958FE99FE02E
:101B80000197F1F700C0000021503109F3CF81E047
:101B90008093E00080E28093D8001092C9008FE12A
:101BA0009EE40197F1F700C0000087E090EBDC01B4
:101BB0008093BA039093BB03A093BC03B093BD037F
:101BC00088E19CE00FB6F894A895809360000FBE62
:101BD00090936000FFCF0F931F93CF93DF938B0100
:101BE000EA0190914C02943051F58093E9008FEF17
:101BF0009091E80095FD06C095ED9A95F1F70000EB
:101C00008A95B1F78091E80085FF19C0ABDE81119C
:101C100011C08091E80085FD06C08091E8008E77B4
:101C20008093E800F3CFF80181918F018093F10058
:101C3000219779F78091E8008E778093E800DF9113
:101C4000CF911F910F910895792F603229F440E2CE
:101C500050E0682F82E0BFCF0895CF93DF93D82F55
:101C6000C92F48E050E0682F792F81E0B4DF88E089
:101C7000ED2FFC2FA0EFB1E001900D928A95E1F7D6
:101C8000DF91CF910895BC0140E250E084E0A3CF02
:101C9000BC0146E050E084E09ECFBC0143E050E050
:101CA00084E099CFFC016081718184E090E00C9424
:101CB000AD319091B60392FB222720F9281751F0FD
:101CC00080FB92F99093B60385EB93E0EBDF82E023
:101CD0000C94C60508951F93CF93DF93C62F122F40
:101CE000632F8430D0F4C530C0F44031B0F490E2BA
:101CF000C99FE0011124C40FD11DC40FD11D90EA6A
:101D0000899FC00DD11D1124CE0189960E94933167
:101D1000612FCE018A960E949331DF91CF911F915E
:101D2000089580911801813061F58091B50387FF96
:101D300028C03EDC8093C10140E250E063E572E0E0
:101D400080EC91E00E944A31892BD1F080E2E0ECF6
:101D5000F1E0A3E5B2E001900D928A95E1F7E09100
:101D60007302F0917402309759F00480F581E02DF0
:101D7000309731F086E08093C00180EC91E00995C6
:101D8000089516DC8093B80148E050E065E772E002
:101D900088EB91E00E944A31892B91F388E0E8EBCF
:101DA000F1E0A5E7B2E001900D928A95E1F7E091AC
:101DB0007302F0917402309719F30280F381E02DE1
:101DC0003097F1F288EB91E0DACF811519F00E949B
:101DD000E105A7CF0895811531F090913403892B47
:101DE000809334039ECF0895811519F00E94E70572
:101DF00098CF0895811539F0809590913403892307
:101E0000809334038ECF089580911703811521F0BC
:101E100082E2F0DF109217030895CF93C82F811547
:101E2000C1F08CEF8C0F813A80F5809118018130E0
:101E300021F48091B50387FD0EC0EAEBF1E08191BA
:101E4000C817F9F021E0E03CF207C9F78C2F28DB36
:101E500068DFCF910895EC2FE695E695E695F0E0E2
:101E6000E054FE4F828190E04C2F477021E030E03B
:101E700002C0220F331F4A95E2F782239323892B56
:101E800029F38C2F41DB4DDFE1CF80E28C0F8830CE
:101E900048F4C77081E001C0880FCA95EAF70E9434
:101EA000E105D6CF8BE58C0F833030F42C2F2452F4
:101EB000330BC901A5DACDCFE8E5EC0FEB3148F4DF
:101EC000F0E0EE0FFF1FE158FE4F80819181C0DAF4
:101ED000C0CF83E38C0F833108F0BBCF61E08C2F40
:101EE00002DCB7CFCF93DF93EC01805E91090897B6
:101EF00020F06BEE7EE0209711F465EE7EE0CE01DF
:101F00000E943D048C2F89DFDF91CF9108956115E8
:101F100029F0209134032260209334039C01305235
:101F20002115304308F49927DDCF811541F19CEF4D
:101F3000980F913A10F4E8DAF4CE90E2980F9830C6
:101F400050F4877091E001C0990F8A95EAF7892FC4
:101F50000E94E705F1CF9BE5980F933018F480E0DD
:101F600090E04ECA98E5980F9B3118F480E090E01D
:101F70006FCA93E3980F933110F460E0B4CB0895E7
:101F8000CF93DF93EC01D1DFCE01805E91090897FA
:101F900020F06AEF7EE0209711F464EF7EE0CE013E
:101FA0000E943D04DF91CF9108951F93CF93DF935B
:101FB000182FEB0132DF209731F4812FB6DFDF914C
:101FC000CF911F9108958FE99FE00197F1F700C02D
:101FD00000002197F0CF6091AD037091AE0389337B
:101FE00021F06091AB037091AC03DFCFEF92FF92D1
:101FF0000F931F93CF93DF93C62FD42F122F8115EA
:1020000099F060932803AFDA9093E4018093E301A1
:10201000C77081E001C0880FCA95EAF7D6DECDB758
:10202000DEB7E6E00C9432318091280368132DC0AE
:10203000E090E301F090E40196DA8E199F09883C64
:10204000910518F500E20D0FCD1799F0C770FF2428
:10205000F3948F2D01C0880FCA95EAF7C5DE0830CA
:1020600040F48D2F877001C0FF0C8A95EAF78F2D01
:10207000ACDE812FB0DF083090F6D77081E001C070
:10208000880FDA95EAF7B0DECACFC77081E001C0E9
:10209000880FCA95EAF7F7CF1092310380911801A3
:1020A000813011F58091B50387FF1EC0E2ECF1E0AD
:1020B0008EE1DF011D928A95E9F780E090E0A0D9DA
:1020C00080E090E0C5D9109234032BDE86E0EFEA81
:1020D000F2E0DF011D928A95E9F71092AD021092AD
:1020E000AC021092AE02D6CAEAEBF1E086E0E1CF94
:1020F000D3DF2FEF84E39CE0215080409040E1F754
:1021000000C0000088E19CE00FB6F894A895809389
:1021100060000FBE90936000FFCFCF93DF93D82F66
:10212000C92F20918D02283010F0B6DF20E0E22F79
:10213000F0E0EE0FFF1FE358FD4FD083C1832F5F08
:1021400020938D02DF91CF910895CF93DF93FB0110
:102150008FEF9FEF4430510588F0D081C1819CDF23
:10216000D093B503C3708091B6038C7FC82BC09306
:10217000B60385EB93E096DD80E090E0DF91CF91B0
:102180000895AAE2B0E0E7ECF0E10C94193188EE92
:1021900091E0FC0101962091F100208321E0803F35
:1021A0009207B9F78091E901893009F457C0C8F462
:1021B000823009F4B2C0833009F482C0813081F1E9
:1021C0008091E80083FFE6C08091E8019091E901E9
:1021D0009A3008F0DFC0E92FF0E0E352FE4C0C9497
:1021E000ED308A3009F489C08B3051F78091E801D5
:1021F000813231F78091EC019091ED01892B01F74B
:102200008091E800877F8093E8008DDB81E09091EA
:10221000EA01911101C080E0809318013DDFD0CF29
:102220008091E801813A61F68091E800877F809390
:10223000E8008091EC019091ED01892B59F060E06C
:1022400080E090E070E016DB8091E8008B7780936F
:10225000E800B6CF68E080EF91E0F4CF8091E8012C
:10226000813209F0ADCF8091EC019091ED018D7F2D
:10227000892B09F0A5CF8091E800877F8093E80043
:102280008091E80082FF17C09091F3008091F200E6
:10229000029731F48091F100813011F0863021F401
:1022A0008091F100809317018091E8008B778093F3
:1022B000E80039DB85CF80914C028111E1CF80CFDE
:1022C0008091E801813A09F07BCF8091EC019091F7
:1022D000ED01892B09F074CF8091E800877F80930E
:1022E000E8008091E80080FFFCCF80911801809386
:1022F000F1008091E8008E77DACF8091E801813299
:1023000009F05ECF8091E800877F8093E8000BDBC7
:102310008091EB018093160153CF8091E801813ABF
:1023200009F04ECF8091E800877F8093E80080918C
:10233000E80080FFFCCF80911601D9CF803889F06A
:10234000823841F58091EC018F70873018F58093C9
:10235000E9008091EB0085FB882780F91092E90065
:1023600006C080912B02880F9091E501892B9091F6
:10237000E800977F9093E8008093F1001092F100BD
:102380008091E8008E7723C0811116C08091EA0108
:10239000813009F18091E80083FF0AC08091E80054
:1023A000877F8093E8008091EB0080628093EB0050
:1023B000AA96E3E00C943531823061F78091EA010E
:1023C000811581F01092E9008091E800877F809369
:1023D000E800A9DADFCF81E0933009F080E0809354
:1023E0002B02F0CF8091EC018F702FEF280F263059
:1023F00088F68093E9002091EB0020FFE3CF933033
:1024000031F48091EB0080628093EB00DBCF909100
:10241000EB0090619093EB0021E030E0A90102C055
:10242000440F551F8A95E2F74093EA001092EA00A4
:102430008091EB008860E8CF8111ACCF1091EA0168
:102440001F778091E3008078812B8093E300809157
:10245000E800877F8093E80066DA8091E80080FFDB
:10246000FCCF8091E30080688093E30083E011114A
:1024700001C082E080934C028DCF8058823008F0FA
:1024800089CF8091EA019091EB018C3D53E0950753
:1024900091F583E08A838AE289834FB7F894DE015D
:1024A000139620E03EE051E2E32FF0E05093570016
:1024B000849120FF03C082958F703F5F8F708A30B8
:1024C000C0F0895C90E08D939D932F5F243161F77C
:1024D0004FBF8091E800877F8093E8006AE270E058
:1024E000CE010196C7D98091E8008B778093E800F0
:1024F00051CF805DE7CF292F33272330310509F4F1
:102500004EC078F52130310509F488C08BE590E0A4
:10251000E8E7F2E02230310509F03CCF2091E800F5
:10252000277F2093E8002091EE013091EF01821780
:10253000930708F49C0140E02115310509F073C0B0
:10254000411171C08091E80082FDCDCF80914C0295
:10255000811549F2853039F28091E80083FFF2CF8E
:10256000C2CF8091EC019091ED012132310509F447
:1025700046C02232310509F00DCF8330910508F0B5
:1025800009CFFC01EE0FFF1FE85DFE4F0190F081C7
:10259000E02D8B5D9E4FDC018C9190E010C09C0182
:1025A0003327823021F12330310568F4232BB9F42D
:1025B000EFE1F3E0E4918E2F90E0EFE1F3E000979C
:1025C00009F4E8CEABCF2330310509F0E3CEE5EED8
:1025D000F2E0E4918E2F90E0E5EEF2E0F0CFE3E15F
:1025E000F3E0E4918E2F90E0E3E1F3E0E8CFE3E065
:1025F000F3E0E4918E2F90E0E3E0F3E0E0CF83306E
:10260000910508F0C7CEFC01EE0FFF1FE25DFE4F03
:102610000190F081E02D89E090E080CF82E190E0B0
:10262000E3EDF2E07BCF80914C02811509F45BCFA2
:10263000853009F458CF8091E80083FD54CF809114
:10264000E80082FD7FCF8091E80080FF75CF9091F8
:10265000F3008091F2002115310519F088309105C1
:1026600050F041E0089709F040E08091E8008E7753
:102670008093E80061CF44914093F100319621505E
:1026800031090196E8CF803809F084CE8091E800C6
:10269000877F8093E8008091E6018093F10070CEFF
:1026A000811178CE1091EA01123008F073CE80913A
:1026B000E800877F8093E8001093E60134D9111574
:1026C000D9F084E080934C0242E061EC81E0A8D92B
:1026D00042E261EC84E0A4D942E261EC82E0A0D95C
:1026E00042E260EC83E09CD980914C02843051F44A
:1026F00082E0809319014ECE8091E30087FDE1CF07
:1027000081E0E0CF81E0F5CF80911A01877F80934F
:102710001A0180911703811105C0809134038D7FC8
:102720008093340380911A0184FF06C08F7E8093CA
:102730001A0182E00E94E10580911A0185FF06C01E
:102740008F7D80931A0180E20E94E105EACACF9250
:10275000DF92FF920F931F93CF93DF93EC018B01D6
:10276000F42E80911A0182FF61C0C0901D03D090A9
:102770001E03CC16DD0619F0209709F057C0809192
:102780001A018B7F80931A01C1E081FD10C08091F6
:102790001B0390911C039801281B390BC1E0809109
:1027A0001001909111012817390708F4C0E08091B9
:1027B0001A01C0FB81F980931A016C2FC6010E9497
:1027C000DE088091310381FF08C080911A01806189
:1027D00080931A0182E00E94E7058091310385FF12
:1027E00008C080911A01806280931A0180E20E94E1
:1027F000E7056C2FC6018BDBF11431F08091A80343
:1028000085FF02C086FF25C08091AB039091AC0389
:10281000B0D980911D0390911E039C013052211567
:10282000304308F49927ACDB6FDF0FC0CE01905224
:1028300081159043B0F4CE019927A2DB80911D034E
:1028400090911E03C817D90779F310931C030093C6
:102850001B03DF91CF911F910F91FF90DF90CF90DD
:102860000895CE01EACF0F931F93CF93DF930DE826
:1028700013E0C9EAD2E0CE010E947731F8016191FC
:102880008F01681719F0CE010E9493312196C13D46
:10289000F2E0DF0781F7DF91CF911F910F9108954B
:1028A0000F931F93CF93DF930DE813E0C9EAD2E0B3
:1028B000CE010E947731F80181938F012196C13DAD
:1028C000F2E0DF07A9F7CDE6D4E0FE01859195910E
:1028D000009711F0FC0109952C96F5E0C53ADF0749
:1028E000A1F7DF91CF911F910F910895EDE8F3E0EB
:1028F000128E138E8FEA90E09183808325E0248FDF
:1029000088E893E1938382838AE090E095838483CF
:1029100044E150E05783468348E050E051874087C8
:10292000938782876EE170E07587648797878687D3
:1029300080E590E0918B808B538B428B48E250E096
:10294000558B448B42E350E0578B468B48EC50E06C
:10295000518F408F158E55A344A3178E168E91A3C9
:1029600080A322A317A216A27EDF96DB1092B603E5
:102970001092B50380E084608093B60385EB93E00A
:1029800091D98ECF0F931F93CF93DF93843028F587
:10299000653018F5403108F520E2629FE00111240E
:1029A000C40FD11DC40FD11D30EA839FC00DD11DAE
:1029B0001124CE0189960E947731082F10E0102F44
:1029C0000027CE018A960E9477319801282BC901F1
:1029D000DF91CF911F910F91089580E090E0F8CFA3
:1029E000462F672F20914F0230915002232B81F404
:1029F000703F39F4403F61F480914D0290914E0256
:102A00000895753028F4403118F4843008F4BACFB2
:102A100080E090E00895A0E0B0E0E1E1F5E10C9401
:102A200015317C010091300380912F03082BC3E006
:102A3000D0E010E0C8010C2E02C0959587950A944D
:102A4000E2F780FD09C02197A8F7D12C8D2DCDB7D5
:102A5000DEB7E7E00C943131DC2EB7018C2FC0DFFC
:102A60000E94ED06019779F3F1CFCF93DF93D82F32
:102A7000C92FD1DF6D2F7C2FB3DF0E94ED06DF91D0
:102A8000CF910895FC018481811561F08781908543
:102A9000009721F00E94ED060C947F0480819181C3
:102AA000E4DFFACF80E008951F93CF93DF93182FD0
:102AB000D92F611589F0411579F0ADDFC82F682F46
:102AC000812F9D2F0E94C104612F7D2F8C2F88DFC5
:102AD000DF91CF911F9108950E94F404C82FF4CF85
:102AE000FC01462F87819085009721F465818081C4
:102AF0009181DACF0895382F292FCB01A32FB22F40
:102B00008F3F9105A105B10520F48F5F9C4F0C9478
:102B1000773180E0089585E290E00E947731823835
:102B200089F486E290E00E947731863359F487E297
:102B300090E00E94773191E0823909F090E0892F8E
:102B40008170089580E0FCCFA6E0B0E0EAEAF5E10C
:102B50000C94153101EC12E081EDE82E82E0F82EA4
:102B600098E0D92E46E050E0B701CE0101960E94D0
:102B70006731F8018D2D11928A95E9F7B8016C5FE4
:102B80007F4F89819A810E940408F8019183808394
:102B9000B8016B5F7F4F8B819C810E940408F80114
:102BA000938382838D8186838E818783F6E0EF0E07
:102BB000F11C085F1F4F81E0E81683E0F80691F6EC
:102BC0002696E7E00C943131A6E0B0E0EAEEF5E1BC
:102BD0000C940F31A0904A02B0904B0281E090E03B
:102BE00090934B0280934A02812C912C10E0640157
:102BF00000E019C021E030E0123020F4F7018591A7
:102C000095919C01472D602F812F65D8739422E008
:102C1000E20EF11C30E17312EDCF0F5F80E1C80EC0
:102C2000D11C053049F0C601880F991FDC01AD5D4C
:102C3000BC4F7D01712CDECF1F5FB0E58B0E911C68
:102C40001430A9F653DEFE01319686E0DF011D92B5
:102C50008A95E9F701ED12E07F0146E050E0B80106
:102C6000C7010E94B1310A5F1F4F0130B3E01B075B
:102C7000A1F7B0924B02A0924A022696EDE00C9486
:102C80002B319C01CB01BA01F9013296E4914E2F10
:102C900050E06E17710548F0F90134966591759111
:102CA0000E94573180E090E008958FEF9FEF0895E4
:102CB000A4E0B0E0EEE5F6E10C9417318B01FC01E5
:102CC0003396F49019821A821B821C82452B31F4B0
:102CD0008FEF9FEF2496E5E00C94333144E050E011
:102CE000BE016F5F7F4FCDDF019691F381E090E0F1
:102CF0000F2C02C0880F991F0A94E2F7092E000CCE
:102D0000AA0BBB0B49815A816B817C81842395235B
:102D1000A623B72321E0892B8A2B8B2B09F420E0F3
:102D2000F801208380E090E0D5CF9C01CA01F90131
:102D30003296E4914E2F50E08E17910550F0F90134
:102D40003496859195910E9457318DDD80E090E019
:102D500008958FEF9FEF0895A4E0B0E0E2EBF6E175
:102D60000C9413317C016B01CA01F7013396B490C6
:102D700019821A821B821C82892B31F48FEF9FEFFC
:102D80002496E9E00C942F3144E050E0BE016F5FDF
:102D90007F4FC70176DF019689F381E090E00B2C2D
:102DA00002C0880F991F0A94E2F780959095092E2A
:102DB000000CAA0BBB0B49815A816B817C81842357
:102DC0009523A623B723F6012081022F017010E07E
:102DD0000B2C02C0000F111F0A94E2F7012E000C09
:102DE000220B330B802B912BA22BB32B89839A833D
:102DF000AB83BC8344E050E0BE016F5F7F4FC701EF
:102E000094DFBECFAAE0B0E0E8E0F7E10C940E3129
:102E1000FE0131968AE0DF011D928A95E9F794E37D
:102E2000A92E91E0B92E8F013F01EE24E394F12CFD
:102E300039E4C32E31E0D32EF50181915F018F3F3C
:102E400009F444C0F894E82FE295EF70F0E021A176
:102E50008F70A70102C0440F551F8A95E2F7CA017F
:102E6000922F982B91A392A18095892382A3789485
:102E700000C0E9E3F1E021E030E0812C912C4191A8
:102E80004F3F79F0A42FA295AF70A05EB0E08C9177
:102E900090E04F7002C0959587954A95E2F780FFC4
:102EA0003BC080E090E0882A992A220F331FCE167B
:102EB000DF0629F7F50182918F3F11F00E94EB07A1
:102EC00050EA5A95F1F7D8018D929C920E5F1F4FF0
:102ED000B9E3AB16B1E0BB0609F0AECF4AE050E073
:102EE000B30180E292E00E944A31892BB9F08AE076
:102EF000F301A0E2B2E001900D928A95E1F781E042
:102F00008093E2010E94B30A9093E1018093E00173
:102F10002A96EEE00C942A31C901C5CF8091E201D6
:102F20008115B1F30091E0011091E1010E94B30A13
:102F3000801B910B059760F34AE050E060E272E07D
:102F400080E492E00E944A31892B49F08AE0E0E275
:102F5000F2E0A0E4B2E001900D928A95E1F71092C0
:102F6000E201D6CFA0E1B0E0E8EBF7E10C940C3140
:102F7000FE01319680E1DF011D928A95E9F700E1BB
:102F800010E0AA24A39493E0B92E412C512C3201D5
:102F90004A944F0173016201B1E14B16510461047F
:102FA00071041CF080E1C82ED12CA601B501C4012A
:102FB0000E948431AC0CBD1C0D2C000CEE08FF08E7
:102FC0004C185D086E087F080150104019F7609694
:102FD000E0E10C9428316FEF85E290E00E9493319C
:102FE0006FEF86E290E00E9493316FEF87E290E00E
:102FF0000E94933160E088E290E00E949331E4DD2A
:10300000B1DF62E885E290E00E94933166E386E2F8
:1030100090E00E94933162E987E290E00C94933152
:10302000A0E0B0E0E6E1F8E10C941331EC01888116
:103030008115F1F0813009F042C08981813029F495
:103040008A8123960E94EB0FF2CF823029F48A8185
:1030500023960E940D0FEBCF833029F48A812396AB
:103060000E94950FE4CF843041F022968111DFCF8A
:10307000CDB7DEB7E9E00C942F318A81239620E0AA
:1030800030E09AE0682F6053770BAB016A3071052E
:1030900060F02115310551F3EFE9FFE03197F1F7C9
:1030A00000C0000021503109F4CF929FB001939FDE
:1030B000700D11249A01260F371F8991E3CFE82F55
:1030C000F0E0E850FE4FB490282F269526952695DF
:1030D00030E0F901E851FE4FE4908770F12C082EA2
:1030E00002C0F594E7940A94E2F7E0FAEE24FF2494
:1030F000E0F8F901E852FE4FC490D12C082E02C02E
:10310000D594C7940A94E2F7C0FACC24DD24C0F821
:10311000F901E853FE4F049110E002C015950795A0
:103120008A95E2F701701127E114F10419F081EE9C
:103130000E940D0FC114D10419F086EE0E940D0FEC
:1031400060E070E08B2D0E94D50FC114D10419F0FE
:1031500086EE0E94950FE114F10419F081EE0E94B1
:10316000950F0115110519F08CE20E94EB0F2196C5
:103170005ECFABE0B0E0EFEBF8E10C940A318C01EC
:10318000DC0114968C91811509F419C160E0C80125
:10319000A7DC9C01F8018681803170F440913B03EB
:1031A00090913A03491333C090918903911521F00E
:1031B00090918A03903158F1D80115969C91911104
:1031C00010C02115B0E53B0708F05BC02115E0E217
:1031D0003E0708F06BC0283E310590F4203E3105D3
:1031E000B0F43093B6022093B502D80112968D91B7
:1031F0009C91909339038093380310921B0107C070
:10320000C9019A9581159F4160F72111EACF61E0CC
:10321000C80166DC7C018091160381114DC0F80164
:103220008581811509F47FC0E114F0E5FF0608F0FF
:1032300064C0E11420E2F20608F0C5C0E11437E0F2
:10324000F306D1F1A8F5C701805E91090897A0F1B6
:10325000309131038091340320912D0399E0F801DE
:10326000A2E0B3E001900D929A95E1F7F0920A0383
:10327000E092090310920C03832B822B80930103AD
:103280001BC0203E42E5340760F4203852E5350784
:1032900008F0BDCFC90180529245809708F0A1CFB8
:1032A000B6CFC90187579C470297F8CF8031F6CF38
:1032B000E1145FE0F50661F6F8014581411185C131
:1032C00023E7E2162CE7F20609F469C0A2EAEA163F
:1032D000A2E5FA0609F497C208F06CC2C701905241
:1032E0008115904208F481C2B1EEEB16F10409F4A5
:1032F0008AC2E5EEEE16F10461C290EEE91692E59F
:10330000F90650F4A0E6EA16A2E5FA06A8F6C70107
:103310009255803491059BCF970127573C47253024
:10332000310508F095CFF9E7EF16FCE7FF0609F045
:103330004EC02091090330910A03232B81F181159E
:10334000A1F081E00E94CB09809101030E94EB0E65
:1033500089E0E2E0F3E0A8EBB2E001900D928A95FB
:10336000E1F780910C038093B70286E0F801A8EBA7
:10337000B2E001900D928A95E1F78091B7028093B7
:10338000160388EB92E0F5DE10921603D80115962D
:103390008C91811104C0809101030E94FA0E8091EA
:1033A00035038770811559F0F8018581811539F051
:1033B0008091B60382FF03C082E00E94C6052B966F
:1033C000E2E10C942631F8018681803140CFBAE7E2
:1033D000EB16BCE7FB0609F06FCF811509F4CAC0F4
:1033E000A0900903B0900A03E0910103E987E98303
:1033F000BE016F5F7F4FC5010E9404082C01F98157
:10340000FB87F1ECCF2EF2E0DF2EEE24E394F12CDB
:1034100022242A94D60117963C90179733FE54C065
:103420006D907C90119712968D909C9013974614F6
:103430005704B9F41496BC91BA87232DF60146813E
:103440006B2F8B850E941E08811559F08A850E947A
:103450006904281634F4D60115969C917401F92A52
:10346000282E48145904C9F431FE17C0F601F5811D
:10347000FA87232DD60116964C916F2F8B850E94CB
:103480001E08811551F08A850E94690428162CF4C3
:10349000F60194817301F92A282E30FE15C0FFEF42
:1034A0002F1212C021E0E216F10471F4232DD6018F
:1034B00016964C9160E08B850E941E08811521F0C4
:1034C000F60185817401F82AF8E0CF0ED11C21E0C5
:1034D00033E02C153D0509F09DCF31E0E316F104F2
:1034E000F1F5998592959F704985942B9F7081E0A5
:1034F000403108F480E0F82EF294E0EFFE22F92A41
:10350000A11450E2B50620F5A11481E0B80608F038
:1035100055C0EA2C8F2D8D704A2D811509F451C0AC
:103520006AE08DEF97E00E94DC09282F30E021153A
:10353000310551F44E2D6EE187ED97E00E94DC09D4
:10354000282F30E0811549F0F901FF297F0107C0DC
:10355000C50190528115904390F1E12CF12C87E048
:10356000EDE0F3E0DF011D928A95E9F7F092150393
:10357000E09214038091140390911503892B09F4B0
:103580000ECFF8018581811539F08FEF0E94CB09AC
:1035900080910C0380930B0386E0F801ADE0B3E06B
:1035A00001900D928A95E1F780910B0380931603A9
:1035B0008DE093E0DEDD10921603F1CEFB28BB24F4
:1035C000A8CF68E085EF97E0AECFC7019757803866
:1035D000910510F00C942423BE2CF0E1EF1608F0B6
:1035E000DECE6EEF70E080E090E085DA8111D7CE1C
:1035F000C12CD12C7601B11042C074E0272EAE014F
:103600004F5F5F4F58874F83AF81B885E22D1D9282
:10361000EA95E9F746015701FFEF8F1A9F0AAF0AB3
:10362000BF0AC701B60167DA8983811509F4B7CEED
:10363000813009F0ABC02601370122E0420E511C57
:10364000611C711CC501B40156DA382E8A838115BC
:1036500009F4A5CE8FEF830D833020F5C301B201AD
:103660004ADA8B83811519F0CE010196D9DC460127
:10367000570133E0830E911CA11CB11C50C02FEFE9
:10368000C216D104E104F10409F489CEC701B601E0
:1036900032DA3FEFC31AD30AE30AF30A8111EFCFFC
:1036A000BA94A9CF8BEF830D8330E0F54601570123
:1036B00043E0840E911CA11CB11CC301B2011BDAB2
:1036C0008B83811561F1C501B40115DA8C838115F5
:1036D000F9F0AB80BC8051E0A5165FEFB50610F0A5
:1036E000BA2CAA2486E0381681F097E0391649F002
:1036F000C5010E9472288091AB039091AC030E9497
:10370000B90DC5010E94932803C0C5010E9472280B
:103710004601570154E0850E911CA11CB11C750196
:10372000640172CFA4E0530142013A12F8CFC30101
:10373000B201E1D9782E46015701B4E08B0E911CFD
:10374000A11CB11CC701B6016D5F7F4F8F4F9F4F0A
:10375000D2D9711409F423CE811509F420CE8150F9
:10376000990B4FEF489F9001499F300D1124E72D91
:10377000E150FF0B2E0F3F1F2150310980F28FE9DE
:103780009FE00197F1F700C00000F6CFCE0101964F
:1037900047DCC5CF109231030E94EF050E94B30AA7
:1037A00088579C4E909319038093180381E080936F
:1037B0001703F5CDF2EBEF16F2E5FF06E9F525EE7E
:1037C00030E02770332781E090E001C0880F2A9510
:1037D000EAF720911A03309117033115E1F04115F2
:1037E000A9F0282B20931A03DACDD80116968C91D4
:1037F000803110F58F2D99278F719927823091058F
:1038000011F04297DBCF21EE30E0DBCF80958223B1
:1038100080931A03C4CD322F3823311569F0982FC5
:103820009095922390931A030E94E705D80115966C
:103830008C91811509F4B3CD80911703811509F49A
:103840007EC0C0903103D0902D030E94B30A8857E8
:103850009C4E9093190380931803F801858181157C
:1038600009F46DC08D2D8C298D798111C7C0E114AB
:10387000F0E5FF06C0F5E11420E4F20608F0C5C04B
:1038800036EEE316F10409F45AC0C70190528115CF
:10389000904208F041C0D80116968C91803108F40E
:1038A000A6C0C701992720911A0120FFB8C02DEFAB
:1038B0002095309134032323209334038D329105D6
:1038C00071F008F0BDC08832910508F0AAC08E31B1
:1038D000910508F0A8C004974A9708F08FC082E0CD
:1038E00080933403A0C0B0EEEB16B2E5FB06E0F423
:1038F000E0ECEE16E2E5FE0610F5F0EAEF16F2E572
:10390000FF0660F420E6E21622E5F206C0F4C701E5
:1039100092558034910598F0C701C5CF34EBE3167A
:1039200032E5F30661F0F8CF49E7E4164CE7F40618
:1039300008F058C057E7E5165CE7F50668F3809194
:10394000A80380FFDBC00E94B30A5C01F8018581F7
:10395000811509F4E4C080911A0182FF06C040E09D
:10396000B50180E090E00E94A713F4E1EF16FCE7B8
:10397000FF0609F4D0C025E1E2162CE7F20609F4AF
:1039800065C033E1E3163CE7F30609F4A9C0C701BB
:1039900090528115904308F063C010921E0310925C
:1039A0001D03D80115969C91911509F41EC2109221
:1039B0002803970130572332310508F016C284E0FE
:1039C00090E00E947F319093B6038093B503F70196
:1039D000E150F047E232F10508F051C1E951FE4CE7
:1039E0000C94ED308BE7E8168CE7F8069BCF8F2D13
:1039F0008F71843109F4A3CF863171F00E94040FD6
:103A000080911A030E94E1059ACFD80116968C91F5
:103A1000803108F046CF93CF86EE92E144CF2FEF6E
:103A200047CF8A9759F780911A03811531F0809119
:103A3000340392E08927809334030E94910E7FCF54
:103A40008C34910581F38D329240ECCF90911A0124
:103A5000892F8E7F90FF816080931A010E948413CA
:103A600080911A0180FF4AC0B8E2EB16F10408F019
:103A70006EC0EEE1EE16F10408F07EC0C7010497B7
:103A80004A9798F58091A80384FD2FC0D801159618
:103A90008C91811509F4D0C09091310380912D0350
:103AA000D82ED92A2D2D2D7F211509F46AC0109208
:103AB0001E0310921D032091A80321FD62C060E047
:103AC000C7010E94DE0860E0C7010E94870F809155
:103AD0002D038D7F0E94370B82E00E94C6055FCCCC
:103AE00080911A01816080931A01D80115968C91FA
:103AF000811521F010921E0310921D03F80185819B
:103B0000F701E851FC47E730F10508F04ACFE75FDD
:103B1000FD4C0C94ED3080911A018E7F9DCF8091E9
:103B20001A018F7E51EEE516F10439F085EEE816A4
:103B3000F10431F480911A018F7D80931A0190CFA6
:103B4000C70190528115904308F08ACF2ACFF9E33C
:103B5000EF16F10468F42DE2E216F10420F43BE2E2
:103B6000E316F10411F68091A80382FDBECF8ECF3B
:103B700044E6E416F104F6CF8091A80383FDB5CFA7
:103B800085CF29E0F801AFE1B3E001900D922A95CD
:103B9000E1F7109222031092210380901D03909070
:103BA0001E03E814F90491F52091A80325FF2EC007
:103BB00030911A0131FBCC24C0F831FF02C026FF3E
:103BC00025C020911B0330911C03F501E21BF30B70
:103BD000E83CF105D8F491FF08C080911A0180619A
:103BE00080931A0182E00E94E7058091310385FFEE
:103BF00008C080911A01806280931A0180E20E94BD
:103C0000E7056C2DC4010E94870FC9CB8D7F0E94F0
:103C1000370BF0921E03E0921D03B0921C03A0929A
:103C20001B038D2D8270846090911A01997FD82E8C
:103C3000D92AD0921A0150CF40E0B501C7010E94A5
:103C4000A713ADCB26E241EE61EE0E94F60FA7CBA3
:103C500027E245EE65EEF9CF26E241EE60EEF5CFC4
:103C600027E245EE64EEF1CF26E241EE62EEEDCFC3
:103C700027E245EE66EEE9CF28E241E0EBCF809106
:103C8000B50381608093B50385EB93E00E94520EEB
:103C90000E944C1084CB8091B60388608093B60359
:103CA000F3CF8091B5038260EDCF8091B50384603E
:103CB000E9CF8091B5038860E5CF8091B60381603C
:103CC000EDCF8091B6038260E9CF8091B50380612A
:103CD000D9CF8091B5038062D5CF8091B503806440
:103CE000D1CF0E944C108091B5038068CBCF8091DA
:103CF000B5038C60C7CF8091B6038360CFCF80912E
:103D0000B5038E7FBFCF8091B603877FC7CF8091E9
:103D1000B5038D7FB7CF8091B5038B7FB3CF8091F3
:103D2000B503877FAFCF8091B6038E7FB7CF8091E9
:103D3000B6038D7FB3CF8091B5038F7EA3CF8091E3
:103D4000B5038F7D9FCF8091B5038F7B9BCF0E9462
:103D50004C108091B5038F7795CF8091B503837F09
:103D600091CF8091B6038C7F99CF8091B50399272D
:103D700082FF939590FB82F990FB83F983CF80912A
:103D8000B603982F909590FB80F990FB81F986CF30
:103D90009091B503892F8F7B96FF806473CF0E942B
:103DA0004C109091B503892F97FB87F980586ACF03
:103DB00061E08EE090E00E94933166CF60E0F9CF41
:103DC0009091B503892F8F7E94FF80615BCF909196
:103DD000B503892F8E7F90FF816054CF9091B603F9
:103DE000892F877F93FF886059CFB6E1EB16BCE738
:103DF000FB06D1F5809131033091A70330FF04C059
:103E0000282F2474211124C0282F2A7A31FF04C0BE
:103E1000482F4171411120E032FF04C0482F4878FB
:103E2000411120E033FF03C08272811120E091151F
:103E300089F081E0211101C080E08093290385E3AE
:103E4000211101C089E20E94500A0E94910EA7CA66
:103E500020E0DCCF80912903811521F085E30E94C9
:103E6000840AF3CF89E2FBCFE7E7EE16ECE7FE0624
:103E700009F1F8E7EF16FCE7FF0639F19701205E3C
:103E800032452032310530F5911124C02E2D2F718D
:103E900081E090E0AC0102C0440F551F2A95E2F783
:103EA0007A01642F83E090E00E9493318E2D0E946E
:103EB000A30475CA81E0911551F00E94A90443E062
:103EC00062E081E00E9427056ACA82E0F4CF0E9486
:103ED000B304F5CF40912A0380913003282F30E0BE
:103EE0002095309570E024233723232B19F04823A5
:103EF00040932A035BE7E5165CE7F50641F491156C
:103F000009F44DCA0E946C040E94040948CA80E466
:103F1000E81682E5F80608F05AC0A0E2EA16A2E523
:103F2000FA0608F05BC0E114B0E5FB0670F5E11499
:103F3000E0E4FE0608F068C0911509F47EC0BAE519
:103F4000EB16BCE7FB0609F4E4C008F0C6C0F1E0DC
:103F5000EF16FCE7FF0609F4DAC023E0E2162CE7CF
:103F6000F20609F4CEC0E1143CE7F30609F065C09F
:103F70000E944C108FEF94E3ACE081509040A04041
:103F8000E1F700C000000E94C70D970130552115D0
:103F9000324090F6970145E0369527954A95E1F72E
:103FA000822F8F7020912A0330E041E050E0082EEC
:103FB00002C0440F551F0A94E2F724233523232B14
:103FC00009F4BACF9111A0CF109231033ECF9701DF
:103FD000205C32452032310508F0AECF8E2D8F7136
:103FE00020912A0330E041E050E0082E02C0440F47
:103FF000551F0A94E2F724233523232B09F49CCF81
:10400000911509F4CCC980CFD80116968C918031D6
:1040100008F092CF911111C02F2D2F7081E090E008
:1040200002C0880F991F2A95E2F720912A0330E0F9
:1040300082239323892B09F0B2C9D80117968D9159
:104040009C91009709F469C00E94ED06F82ED92EC4
:1040500086E0F801DE01119601900D928A95E1F754
:10406000D8011596CC9015971696BC90B2942FE077
:10407000B222809135038770811509F1AC2CC114EF
:10408000F9F0892F807F803469F080E28F0D8830CD
:10409000B0F0892F807E803229F4B2E0FB1678F0F0
:1040A000B11469F08091B60382FF09C082E00E94DA
:1040B000C605809135038770AA24A3948111A12C91
:1040C0008D2D82958F70882E912C8C3008F059C0E0
:1040D000F401E05FFD4C0C94ED304BE5E4164CE749
:1040E000F406C9F08091B603002482FF0394802D6A
:1040F0005CE5E5165CE7F50609F09FCF0E94590ED6
:104100009CCF6FEF7FEF80E090E00E94AD310E9486
:10411000781081E0F3CF80E0F1CFF8018581C08095
:10412000D180811569F0C6010E940B15F82E682F09
:10413000C6010E94C104B6018F2D0E94F01484CFE5
:10414000C6010E94F404F82EF6CFED2DEF70EE2E8E
:10415000F0E1DF1618F0E29490EFE922C11409F4BF
:104160004BC0E11459F080E28F0D883010F0F1104F
:104170003DC08E2D0E94E1050E94910E8F2D0E9460
:104180000D0F28E0821A910834E08316910418F488
:104190000E94F109A12C8F2D9D2D0E947F04811575
:1041A00041F0C11409F425C2B11409F419C21092E6
:1041B000B903A114B1F08091350380FD12C0D8017C
:1041C00015961C928695869586950E94A904C8012D
:1041D0000E94B918809135038695869586950E9430
:1041E000B30460E0C8010E947015E9C880913403EF
:1041F0008E2980933403C0CF8F2D0E94950FE11438
:1042000009F4BFCF80E28F0D883010F0F11004C0A8
:104210008E2D0E94E70506C0E094809134038E2124
:10422000809334030E94910EACCF4D2D4F70E42E3D
:104230008D2D807F803219F0E29480EFE822F11416
:1042400051F051E0F51609F473C0C11409F47FC0B0
:10425000B114D9F093CF8091B60382FD12C0C1147E
:1042600049F0E11429F08E2D0E94E1050E94910E83
:1042700080E085CF80E00E94950FE11409F481CFA2
:10428000C7CFC11491F1B11004C08E2D0E94E50E6C
:1042900078CF81E0B81211C070902D038E2D872148
:1042A000E81609F46ECF0E94B30A90932C03809312
:1042B0002B037E2870922D0364CF8091A903823056
:1042C00008F45FCFB8125DCF8E2D0E94E50E8E2DC3
:1042D0000E94220B80912E039E2D9823E91609F44B
:1042E00050CF8E2980932E034CCFB11012C08E2D4B
:1042F0000E94F40E8E2D0E94220B80912E039E2D83
:104300009823911509F43DCFE094E822E0922E0322
:1043100038CF8091A903823008F433CF91E0B912ED
:1043200030CF809131038E21811509F42ACFDFCF60
:104330008091AF03C11421F08B1508F422CFA5CFD3
:10434000B81608F01ECF8E2D0E94F40E1ACFB114AD
:10435000D1F3A9E3FA1609F03BC18091AD03909126
:10436000AE030E94B90D8F2D0E94950F0ACF8D2D9F
:10437000869586958370811569F0813009F001CFAB
:104380008F2D9D2D9370C11002C080E090E00E949F
:10439000280AF7CE8F2D9D2D9370C11002C080E0AA
:1043A00090E00E94000AEDCE6C2D8F2D0E94730BC1
:1043B000E8CE8D2D8370811133C0C110E2CE4F2D18
:1043C000429546954770440F440F8F2D8F70042EF1
:1043D00001C0880F0A94EAF72F2D2071F4FE07C060
:1043E0002FE030E001C0220F4A95EAF720953D2DDD
:1043F000369536953370323071F0333051F040914C
:104400002F03313029F0822B84230E94A304B9CEDC
:10441000842B822BFACF822B90912F038927F5CF03
:10442000C11459F1D0FEADCE4F2D4295469547703F
:10443000440F440F8F2D8F70042E01C0880F0A94F3
:10444000EAF72F2D2071F4FE07C02FE030E001C005
:10445000220F4A95EAF720953D2D36953695337013
:10446000323091F0333071F040913003313049F007
:10447000822B84230E94A60484CE823008F481CE4D
:10448000D3CF842B822BF6CF822B909130038927B8
:10449000F1CFBD2DBF70EB2EC11429F08B2F0E94E0
:1044A000A9048F2DF3CE8F2D0E94F40E8E2D0E9425
:1044B000B30467CEE2EFFE16A1F1F3EFFF1670F43E
:1044C00020EFF216D1F031EFF31691F0C11409F498
:1044D0007AC0B11053CE8D2D8F7127C043EFF416E3
:1044E00039F154EFF512F2CF8091B60382FD2CC062
:1044F0008D2D8F71C114D9F218C08091AF03C114F2
:1045000061F0B81608F03DCE2D2D2F7181E090E0BE
:1045100001C0880F2A95EAF7B8CF8B1508F431CE81
:10452000F3CF8D2D8F71C110C2CF0E94A90429CE67
:1045300080E0C11409F49ECF81E09D2D9F7101C0E0
:10454000880F9A95EAF796CF8091A903823048F1B7
:10455000C114C9F0909135039770943059F41092BA
:10456000350310923703109236038D2D8F710E9400
:10457000B3040ECE63E0B81608F00ACE8D2D8F710D
:104580000E940E0B05CEB81640F010923503109223
:1045900037031092360364E0F1CF81E00E94C60534
:1045A000F7CDC11431F063E08D2D8F710E940E0B99
:1045B000E8CD81E00E94C60582E0B81608F4E1CD9E
:1045C0000E94C605DECDB11441F099E3F916C3CEC1
:1045D0008091AB039091AC03C4CE8D2D8F7167CFCA
:1045E00080913303809332038091310380933303AE
:1045F000E0CD40E060E089819A810E9454159C01E1
:10460000E0903103B11429F01092B903E092330322
:10461000D0CD8091B7039091B80328173907B1F72F
:104620008091AA0382FFF0CF8091B903811561F3D5
:10463000809132030E94E50E8F2D0E94EB0F809136
:1046400032030E94F40EE0CFF3E7EF16FCE7FF061B
:1046500011F00C94661980911703811509F49AC81A
:104660000E94040F0C94CF1980918A03803178F452
:1046700080918903811559F0E0913B0320913A0321
:10468000309185034091840359E02E1301C00895B1
:104690006E2F70E05E9FF0011124DF01A45CBC4F1F
:1046A00014968C911497811559F111968C9111974C
:1046B000831326C08C91841323C015968C91159773
:1046C00081111EC012968D919C91A0918603B0918C
:1046D00087038A1B9B0B883C910590F480918A0389
:1046E0008F70806180938A03EE5BFC4F80818F70B6
:1046F0008061808384E893E00E94B9180C94BC0523
:10470000FB013196E770C1CFCF92DF92FF920F93FA
:104710001F93CF93DF93182F092F89E0F82EC091B4
:104720003B0380913A03C81799F1FC9EE0011124E4
:10473000CE01845C9C4F6C01FC018581811589F060
:10474000C6010E944215811561F0FE01EE5BFC4F2F
:1047500020812F7020612083F601808191810E9449
:104760008D10C6010E94B91820913B0330E02F5FE5
:104770003F4F2770332720933B03C45CDC4F898174
:104780008013CDCF88818113CACF8D81811539F2F5
:10479000DF91CF911F910F91FF90DF90CF900895FF
:1047A000EF92FF921F93CF93DF93EC0120911B01B7
:1047B000211541F010E0812FDF91CF911F91FF90E3
:1047C000EF900895EA80FB80E61AF70A24EFE216DC
:1047D00021E0F20678F760E0CE010E9470159C019E
:1047E00030522115304330F70E948705811511F3AF
:1047F0008091B5029091B6020E948705182F81150D
:10480000C9F28091B3039091B403853F21E09207F0
:1048100010F084EF91E0E816F90660F68E818F7053
:1048200080618E83888199810E948D100E94460547
:10483000CE010E94B918BFCFAFE0B0E0E2E2F4E2EF
:104840000C940C318C0186E0F801DE011A9601907F
:104850000D928A95E1F7D8016C9011965C901197B2
:104860001296AD90BC9013971496EC9014971596F1
:10487000FC90F1100CC050918D02252F30E0E0E04B
:104880008E2F0E2E000C990B821793073CF154E8E3
:10489000C52E53E0D52E80918803811151C0E114BB
:1048A000D1F0F11409F408C3C8010E944215811522
:1048B00009F402C36091380370913903C80170DFB5
:1048C000811109C089E0F801A4E8B3E001900D92DC
:1048D0008A95E1F7C9DEFF24F39486C0880F991FFB
:1048E00083589D4FDC0111964C911197451103C0DF
:1048F0008C91681611F0EF5FC3CFEF3F41F2D80102
:1049000016968C9116978F70806116968C93E5178A
:10491000A0F4AFEFA50FA0938D02EA1770F4F0E0BA
:10492000EE0FFF1FE358FD4FB0E0AA0FBB1FA358C7
:10493000BD4F8D919C91918380830E944605A7CFA6
:1049400060E084E893E00E9470159C0170908903F8
:1049500080918603909187034501881A990A711402
:1049600009F457C2B8EC8B16910408F00DC2E1149B
:1049700009F4B1CF80918503F8019181E0908A0319
:10498000F0E1EF1608F0C6C1981350C0909184036F
:10499000D8018C9198134AC0F11048C08E2D8F70A9
:1049A000806180938A0384E893E00E94B918809123
:1049B0008A03F8018683F0908603E090870349E03C
:1049C000D42E00913B0380913A03081751F0D09EFA
:1049D00080011124045C1C4FD80115968C91811123
:1049E00008C00E94BC05F12C8F2D2F96E0E10C949D
:1049F0002831F801B280C380C8010E94421581119C
:104A00000EC0C8010E94B91880913B0390E0019646
:104A10008770992780933B03FB2CEC2CD2CF6F2D12
:104A20007E2DC801BDDE8111EFCFDBCF30522115C5
:104A3000304308F084C0F11005C140E0652D862D9B
:104A40000E949A0D81114FC040E0652D862D0E9475
:104A50009A0DF82E811509F429C18091AA0380FFCF
:104A6000C2CF84E893E00E94B91860E084E893E044
:104A70000E9470158C01F0903B037F2C98E0E92E8A
:104A800024E8822E23E0922E39E0432E80913A03CF
:104A90007816A1F0A72CB12C479CC0011124FC0171
:104AA000E45CFC4F6F0160E0CF010E947015582E4E
:104AB000692ED60115968C91811197C0B8E0EB163E
:104AC00018F419E0EF10ACC08A859B851DDE0E94AA
:104AD00046050E94BC0589E0E4E8F3E0DF011D9291
:104AE0008A95E9F780CF60E0C8010E947015809137
:104AF000AA0383FFA9CFB80184E893E00E9453057D
:104B00008111A2CF80918A038F70806180938A0384
:104B100080918403909185030E948D1084E893E036
:104B20000E94B918E4E8F3E089E0DF011D928A955C
:104B3000E9F78A859B85E8DD0E94460552CFF1148E
:104B400009F482CF80918A03816080938A038091E7
:104B5000AA0381FF48CF84E893E00E94B91800912E
:104B60003B0380913A03081709F4CCC0E02EF12CE6
:104B7000B9E00B9FC0011124FC01E45CFC4F6F0104
:104B8000CF010E944215811509F4BCC089E0F601ED
:104B9000A4E8B3E001900D928A95E1F7C701019670
:104BA00087709927082F80933B030E94BC0589E0FA
:104BB000F82E80913A03801709F413CFF09E8001FC
:104BC0001124045C1C4FC8010E944215811109CFB9
:104BD000C8010E94B91880913B0390E0019687704C
:104BE0009927082F80933B03E4CF10520115E0E38F
:104BF0001E0708F063CF8091AA0383FD0AC0E72C4B
:104C0000C5010196F82FF7707F2E052D162D460150
:104C10003DCFB601C4010E945305811589F3EFCF42
:104C20001F9DC0011124845C9C4F0E94B9182091E3
:104C30003B0330E02F5F3F4F27703327F22E209346
:104C40003B0340CF80918A03816080938A0360E0B8
:104C5000C8010E9470158091AA0383FF78CFB80124
:104C600084E893E00E945305811171CFF0908A038C
:104C7000E894F0F8F0928A03C8010E94421581116D
:104C8000B2CE8F2D8F70806180938A0380918403D0
:104C9000909185030E948D100E94460584E893E060
:104CA0000E94B918E4E8F3E089E018CF8A859B8573
:104CB0000E943515292F22952F70903450F49F7043
:104CC000223080F0911599F0F8019681903178F4B6
:104CD0008BCE2A5F2F70223078F0C8010E94B9185D
:104CE000F72C82CE911519F0811509F47DCE805EE6
:104CF000883008F479CEF1CF803F08F475CE815F1B
:104D00008330F7CF89E0E4E8F3E0DF011D928A9574
:104D1000E9F74DCF981315C090918403F801808175
:104D200098130FC0F1100DC0E682C8010E94B91897
:104D300089E0F801A4E8B3E001900D928A95E1F7CB
:104D4000CACDC8010E944215811509F4B5C0F114FD
:104D500009F4B2C080918A03803208F4B3CD1E8278
:104D60001F821886198680918403909185039A8307
:104D70008983BC82AB82809188038D83EF82CE01D0
:104D800001960E94B9189ECD90908A03F0E19F167B
:104D900038F484E893E00E94B91889E0D6019FCEE8
:104DA000E11409F498CD90918503F801818198135D
:104DB00011C090918403808198130CC0F1100AC037
:104DC0009682C8010E94B91889E0D6011D928A9581
:104DD000E9F781CDC8010E944215811509F46CC024
:104DE000F11409F469C080918A03803208F46ACD15
:104DF0001E821F82188619868091840390918503F4
:104E00009A838983BC82AB82809188038D839F8241
:104E1000B6CFB8EC8B16910408F052C0E11409F437
:104E20005ACDF11409F448C090918503F8018181AD
:104E300098132AC0909184038081981325C060E064
:104E400084E893E00E9470158091B1039091B203C1
:104E50008816990608F06CCF80918A0380FD68CF90
:104E6000803108F465CFD80116968C931697982F49
:104E7000907F903F09F459CF982F907F905F8F706B
:104E8000892B16968C9351CFC8010E94421581152B
:104E900071F06091380370913903C80181DC81158C
:104EA00009F410CD89E0E4E8F3E0DF018FCF8091D1
:104EB0008A03816080938A03C8010E94B9180BCDD0
:104EC00089E0F60111928A95E9F78DCDA1E2B0E073
:104ED000ECE6F7E20C9416314C8F5D8F6E8F7F8F6E
:104EE000082F88A3192F99A3F82EE92E811509F40C
:104EF000A3C040E0692F8C8D9D8D0E9454159C01AC
:104F0000111549F01092B9039093B8038093B70339
:104F1000109234030AC08091B7039091B8038217AE
:104F2000930719F481E08093B903198E1A8E1B8EB2
:104F300086E0FE017C96DE01539601900D928A95E3
:104F4000E1F78091B60382FF21C080918F03909199
:104F50009003892BD9F00E94B30A20913603309137
:104F60003703821B930B20918F033091900382179C
:104F7000930738F08091350382FD03C082E00E94E0
:104F8000C6050E94BF0A81110E94EF05F11461F06D
:104F90000F8B188F61E0CE0143960E94701561E07F
:104FA000CE0143960E9470150F8B188F89E0FE0189
:104FB0007396DE011A9601900D928A95E1F7CE0163
:104FC0000A963ADC811110C020913A0330913B03DC
:104FD00089E0FE013A96DE01119601900D928A95C4
:104FE000E1F78E8581112CC019E080913B039091EF
:104FF0003A03891741F0189FC0011124845C9C4F2B
:105000001BDC811144C08E85811112C080911B016F
:1050100081110EC08C859D85209138033091390314
:10502000821B930B8F3F9F4318F081E080931B01FD
:10503000A196E6E00C943231911509F476CF68CF51
:10504000822F90E00196877099273817190671F41E
:105050000E944C1010923A0310923B0389E0E4E85E
:10506000F3E0DF011D928A95E9F7BECF99E0929FA8
:10507000D0011124A45CBC4FFE01319601900D9229
:105080009A95E1F780933A030E94BC05ADCF8091D9
:105090003B0390E001968770992780933B03A5CF4F
:1050A000A6E0B0E0E6E5F8E20C9418310E94B30AFD
:1050B0008C0180915102909152028017910771F0FA
:1050C00019821A820E94B30ABC0149815A8180E088
:1050D00090E0FCDE10935202009351022696E4E029
:1050E0000C943431A6E0B0E0E8E7F8E20C941A3111
:1050F00090934E0280934D02811520E2920730F486
:105100000E94720F2696E2E00C94363180EF89837C
:105110008A830E94B30A8160BC0149815A8181E07F
:1051200091E0D4DEEFCFA6E0B0E0E9E9F8E20C943C
:105130001A3190934E0280934D02811520E292071E
:1051400030F40E94C00F2696E2E00C94363180EFD6
:1051500089838A830E94B30A8160BC0149815A8194
:1051600081E090E0B3DEEFCFCDB7DEB7AC970FB6FE
:10517000F894DEBF0FBECDBF85B7806885BF85B709
:10518000806885BF84B7877F84BF0FB6F894A895E1
:1051900080916000886180936000109260000FBE73
:1051A00080E890E00FB6F8948093610090936100DE
:1051B0000FBE81E08093190189EE97E09093B701CB
:1051C0008093B6010E94A4150E9450140E94E30C23
:1051D0000E94400D8091E20084608093E200789408
:1051E00080914C02811599F08091E9001091EC00BA
:1051F0008F70179511271795182B1092E900809141
:10520000E80083FD0E94C1101F701093E90082E046
:1052100084BD93E095BD9AEF97BD80936E000E9488
:105220008B15811102C00E94EB1704E311E0D80135
:105230008D918D018F3F11F00E94EB07B1E0093392
:105240001B07A9F709E311E0E9E4EE2EE1E0FE2EE9
:10525000F80181918F018F3F11F00E94EB07E0165A
:10526000F106B1F78AE0E0E4F2E0DF01282F1D92B9
:105270002A95E9F7E0E2F2E0DF011D928A95E9F76D
:1052800080E090E00E947F31833E9E4F21F40E9497
:105290008B1581112AC063EE7EEF80E090E00E94C2
:1052A000AD3160E082E090E00E94933181E0809334
:1052B0002F0361E083E090E00E949331198284E142
:1052C0008A83CE0101960E94520E0E94EB1740E0A5
:1052D00050E0BA018FE090E00E94A53140E050E03C
:1052E000BA0183E190E00E94A53182E090E0FFD70F
:1052F00080932C0284E090E00E947F319093B6036B
:105300008093B5030E940217EFEFF6E721E0E1502A
:10531000F0402040E1F700C000000E940217809199
:10532000400280FF08C06FEF7FEF80E090E00E94B6
:10533000AD310E94C70D83E090E0D9D70E94A3044D
:1053400084E091E09093740280937302AE014F5F0A
:105350005F4F1A0180914C0210E4853009F48DC032
:105360000E9402177DE2672E72E0772E00E412E0C1
:10537000D801F301219131918D919D9147E352E044
:105380004E175F0709F483C02817390799F360E4C3
:10539000A62E62E0B62E912CD501ED90FD905D0118
:1053A000F301419051903F014E145F0451F14E249E
:1053B0005F24812CCC24C394D12CC2018C219D214B
:1053C000892BB1F089829A820E94B30A9C838B83D5
:1053D000F1E0FD8391E097012C213D21232B09F47D
:1053E00090E09E8349815A816B817C818D816EDD45
:1053F0008394CC0CDD1C20E18212DFCFF301F2920A
:10540000E292939435E09312C7CF0E942E0C44C0D1
:1054100080914C02843019F110922A0288E190E0C8
:105420000FB6F894A895809360000FBE10936000AB
:1054300083B7817F846083BF83B7816083BF7894A3
:10544000889583B78E7F83BF0FB6F894A895809117
:105450006000886180936000109260000FBE0E941F
:105460000217E0E4F2E081919191892B09F0C5C423
:10547000AAE4B2E0AE17BF07B1F780914C028530C5
:1054800009F4C6CF0E944C100E94F10969CF281779
:10549000390709F07CCF04DE8091A80380FF1CC08F
:1054A00080911A0182FF18C00E94B30ABC0180914A
:1054B0001B0390911C039B01281B390B8091100149
:1054C000909111012817390738F041E080911D03B0
:1054D00090911E030E94A71380911703811569F014
:1054E0000E94B30A2091180330911903821B930B79
:1054F0008F3F9F4710F40E94040F86E0EFEAF2E02E
:10550000D10101900D928A95E1F79090B002B09090
:10551000B102C090B202A090B302D090B402109237
:10552000B1021092B2021092B3021092B4028C2D0A
:105530008B298115A1F0E0903902F0903A020E9487
:10554000B30A9C012E193F099091AD02911509F4FF
:105550008DC0809115018217130608F495C08D2D1A
:105560008A298115A1F0E0903702F09038020E945C
:10557000B30A9C012E193F099091AC02911509F4D0
:10558000B3C0809113018217130608F4BBC0809149
:10559000B002891119C08091B102811511F08B11EF
:1055A00013C02091B202211511F02C110DC0909161
:1055B000B402911511F09D1107C03091B302311161
:1055C00003C0822B892B81110E944A0B86E0F101D6
:1055D000AFEAB2E001900D928A95E1F70E94F109DD
:1055E00090913B02891721F080933B020E942E0C80
:1055F00080914C02843009F0ADCE83E08093E900C5
:105600008091E80082FFA6CE8091E80090E085FFBF
:105610000AC00E94B20C30E2E32EF12C6101811528
:1056200009F4AAC091E08091E8008B778093E800AC
:10563000911509F48FCEE0904F02F0905002E9816D
:10564000E114F10409F4A6C0EE3F09F0C5C08A8157
:10565000833020F08550833008F0BEC0EA81EE3000
:1056600008F0BAC0F0E0E45EFD4CB7C5409114010B
:105670008AE0489FA00111244217530708F06FCF1A
:105680009F5F9093AD0202C09F3FD1F7B11459F0D4
:105690000E94390991E01B140CF09FEF899F802D27
:1056A00011248093B102C11459F00E94390991E08C
:1056B0001C140CF09FEF899F802D11248093B2025F
:1056C0008091B102811509F44ACFF090B202F11431
:1056D00009F445CF0E942B098093B1028F2D0E94BF
:1056E0002B098093B2023BCF40911201AAE04A9F5E
:1056F000A00111244217530708F049CF9F5F9093F0
:10570000AC0202C09F3FD1F7A11459F00E94920948
:1057100091E01A140CF09FEF899F802D1124809343
:10572000B302D11459F00E94920991E01D140CF0BB
:105730009FEF899F802D11248093B4028091B30242
:10574000811509F424CFF090B402F11409F41FCFAD
:105750000E942B098093B3028F2D0E942B09809306
:10576000B40215CF8091F100F60181936F01F1E051
:10577000EF1AF10809F456CF8091E80085FDF2CFC9
:105780008091E8008B778093E8000E94B20C81152D
:1057900099F348CFE43148F4E11551F0E150E33199
:1057A00038F4F0E0E65DFD4C18C5EE3F09F456CF45
:1057B0008FEF4FC31A8289E08B830EC08A818230BB
:1057C00079F08330A9F0813099F70E942E0C1BD517
:1057D0006B837C838D839E83C1010E94020DBACDB1
:1057E00088E290E084D51B821C821D828E83F4CFD8
:1057F00080914A0290914B02892B71F3F101D801FB
:105800008C9111969C910E5F1F4F928383833296E9
:10581000B2E00A341B0799F7DFCF8A81823041F664
:105820006B817C818D819E81EED488E290E07BD576
:10583000D3CF4C816B818A810E94C214982789271B
:1058400098279E838D83C8CF2D813E8132272327C1
:1058500032274C816B818A810E946B0EBDCF0E94E2
:10586000E415BACF80E18A83B7CF1A828FEFA4CF35
:105870008C818D3108F0B0CF8A809B809824892458
:105880009824A12CB12C81017101E80EF11CE016C5
:10589000F10609F4A1CF80E0EFEF8E169104A10488
:1058A000B10420F4C4018F5F9C4F21D5D801149618
:1058B0008C930F5F1F4FBFEF8B1A9B0AAB0ABB0A7B
:1058C000E6CF80914A0290914B02892B09F484CF54
:1058D0008C818D3108F080CF882E912CA12CB12C99
:1058E000CA80DB80DC24CD24DC24E12CF12C810176
:1058F000412C512C3201481459046A047B0408F0ED
:105900006BCFEFEFCE16D104E104F10438F4D801E7
:1059100014966C91C6018F5F9C4F05D5BFEF4B1A53
:105920005B0A6B0A7B0AEFEFCE1ADE0AEE0AFE0A6A
:105930000F5F1F4FE0CF0E94B2174ECF84E093CF8E
:105940008C818D3108F048CF882E912CA12CB12C60
:10595000CA80DB80DC24CD24DC24E12CF12C412C1A
:10596000512C32018E010B5F1F4F481459046A04F9
:105970007B0408F031CF80E0F0E8CF16F2E0DF06DC
:10598000E104F10418F4C6018996B1D4D8018D93CD
:105990008D01BFEF4B1A5B0A6B0A7B0AEFEFCE1A41
:1059A000DE0AEE0AFE0AE1CF2C81022F10E02D3133
:1059B00008F012CF8A819B819827892798272C018C
:1059C000612C712C8038F2E09F0708F005CF822E01
:1059D000912CA12CB12C40E852E060E070E0441919
:1059E000550966097709421751056105710508F4E3
:1059F000F3CE20914A0230914B02232B09F03FC095
:105A00009C01275D3F4F3CA72BA780FBEE24FF2482
:105A1000E0F880FF0BC088966AD49D81892798277B
:105A2000892781159C4711F48FEF8D83D501C4011F
:105A3000840D951DA61DB71D80FF1AC0680141E0A9
:105A4000C41AD108CE0105968C0D9D1D9AA789A771
:105A50008BA59CA5800F911F4AD4A9A5BAA59C919E
:105A600081159C4721F48FEFE9A5FAA58083860173
:105A7000F101EE0DFF1D2FEFE016F10628F0810178
:105A8000C12CD12C760125C09481858181159C473C
:105A900011F42483258342E0E40EF11C3296ECCF0E
:105AA00050E8451652E055066104710430F4D801FF
:105AB00014966C91C201899636D4BFEFCB1ADB0ADB
:105AC000EB0AFB0AEFEF4E1A5E0A6E0A7E0A0F5FC0
:105AD0001F4FC814D904EA04FB0410F37DCE809153
:105AE0004A0290914B02892B09F476CEC1010E94A3
:105AF000020DFFEF21EE34E0F15020403040E1F79D
:105B000000C0000016CC88E0ECE1F1E0DE019196E7
:105B100001900D928A95E1F7FE0132968FE1DF0147
:105B20001D928A95E9F786E0898388E07F96DE01F9
:105B3000159601900D928A95E1F74ECE8CEE8983F1
:105B400081E08A831B821C8247CE8B819C81092E37
:105B5000000CAA0BBB0B25E0880F991FAA1FBB1FC7
:105B60002A95D1F7AC01BD01405E5F4F6F4F7F4F6B
:105B7000481759076A077B0708F42ECE8C3EE1E0F0
:105B80009E07A105B10508F027CE4D3EF1E05F0765
:105B90006105710520F04CEE51E060E070E0481BBB
:105BA000590BBC0165567A4FC1016BD315CE4AE142
:105BB00050E06FEF70E0CE01079682D380914A02E9
:105BC0008983EA821B821C8282E08D838DE00ECE67
:105BD00081E090E09093500280934F0282E390E046
:105BE00090933F0280933E020E94B30A90933D023D
:105BF00080933C02F1CDE114F10481F1D090400298
:105C0000C090450200913C0210913D020E94B30AEF
:105C1000801B910B8536910540F1C5FE26C0D0FE54
:105C200024C00E94B30A90933D0280933C0280916D
:105C30003E0290913F02019790933F0280933E0273
:105C4000892B61F41092500210924F0281E090E093
:105C500090934B0280934A02E12CF12C80914A02EE
:105C60008983EA8280913E02A7CD82E390E09093FF
:105C70003F0280933E02F2CF10924B0210924A02F2
:105C8000ABCD0B811C8140E250E06FEF70E0C101B1
:105C900017D323E634E042E050E080E090E0F901E1
:105CA000659175910617170730F4820D931DDC017D
:105CB0006D937C93CA01B5E02F383B0709F48CCD76
:105CC000AC014E5F5F4F245F3F4F4132510538F3C7
:105CD00083CD2B813C8183E694E0FC014591559175
:105CE0002417350709F4A6C00C96E5E08B399E070A
:105CF000A1F75ECD8B819C8103E614E0F80125912C
:105D000035918217930709F4A6C0045F1F4FF5E091
:105D10000B391F0799F7EE24EA94FE2CB7C00E94B6
:105D200076145ACD8B81873071F0883049F181111A
:105D300053CD8FE1D1011D928A95E9F788E08C83DC
:105D400083E088A349CD2C8166E0CE018196FC01D9
:105D5000362F11923A95E9F7283080F4629FB0010E
:105D600011246F527D4F46E050E0B1D280E089832C
:105D700086E0FE01B196DE011296DBCE8FEFF7CF03
:105D80006C8186E0FE013596DE01919601900D92C0
:105D90008A95E1F789A19AA181154CE7940741F40E
:105DA00020914A0230914B02232B11F480E090E0C5
:105DB0009AA389A38BA19CA181155CE7950741F467
:105DC00020914A0230914B02232B11F480E090E0A5
:105DD0009CA38BA38FEF683060F486E0689FB001CE
:105DE00011246F527D4F46E050E0CE018196B9D22A
:105DF00080E089830E94A415EFCC80912B0281154D
:105E000009F43BCBB0E1B9BDE2E1E9BD09B400FE64
:105E1000FDCF8091D8008F7D8093D8008091E000E5
:105E200082608093E0008091E00081FDFCCF0E94C1
:105E30004C1023CBFC013696259135912115310567
:105E400009F4B6CC4FE150E0BE016E5F7F4FF9011F
:105E500009958983C1CCF801389625913591211592
:105E6000310509F458CF4CE150E0BE016B5F7F4F24
:105E7000C801F90109957C01892B41F4F8013A9692
:105E800085919591009711F0FC010995E982A4CCC8
:105E90001F921FB61F9211248F939F93AF93BF93AE
:105EA00080912A02811113C08091F8019091F9012B
:105EB000A091FA01B091FB014196A11DB11D809303
:105EC000F8019093F901A093FA01B093FB01BF91FF
:105ED000AF919F918F911F901FBE1F90189578943E
:105EE0001F921FB61F9211248F939F93AF93BF935E
:105EF0008091F8019091F901A091FA01B091FB0114
:105F00000196A11DB11D8093F8019093F901A09312
:105F1000FA01B093FB01BF91AF919F918F911F90B8
:105F20001FBE1F9018951F920F920FB60F9211244B
:105F30002F933F934F935F936F937F938F939F9391
:105F4000AF93BF93EF93FF938091E10082FF09C06D
:105F50008091E20082FF05C08091E1008B7F8093F9
:105F6000E1008091DA0080FF24C08091D80080FF9A
:105F700020C08091DA008E7F8093DA008091D90072
:105F800080FFA9C080E189BD82E189BD09B400FE1E
:105F9000FDCF81E080934C028091E701811109C01F
:105FA0000E94E30C0E94400D8091E2008460809387
:105FB000E2008091E10080FF1AC08091E20080FF42
:105FC00016C08091E2008E7F8093E2008091E20013
:105FD00080618093E2008091D80080628093D80035
:105FE00019BC85E080934C0283E080931901809175
:105FF000E10084FF2FC08091E20084FF2BC080E18C
:1060000089BD82E189BD09B400FEFDCF8091D80031
:106010008F7D8093D8008091E1008F7E8093E10096
:106020008091E2008F7E8093E2008091E2008160A7
:106030008093E2008091E601811509F452C084E06A
:1060400080934C0280914C02843009F052C082E06F
:10605000809319018091E10083FF2CC08091E200C0
:1060600083FF28C08091E100877F8093E10082E078
:1060700080934C021092E6018091E1008E7F809324
:10608000E1008091E2008E7F8093E2008091E20047
:1060900080618093E20042E060E080E00E94100DA9
:1060A0008091F00088608093F00081E08093190176
:1060B00080931801FF91EF91BF91AF919F918F91C4
:1060C0007F916F915F914F913F912F910F900FBEF4
:1060D0000F901F90189519BC10924C021092E70176
:1060E00068CF8091E30087FF02C083E0A9CF81E001
:1060F000A7CF81E0ADCF1F920F920FB60F92112460
:10610000EF92FF920F931F932F933F934F935F93C1
:106110006F937F938F939F93AF93BF93CF93EF939F
:10612000FF9309EE10E0F8018081C091EC008F70C0
:10613000C795CC27C795C82B108280EFE82EF12C8D
:10614000F7018081877F808378940E94C110F801D5
:106150001082F701808188608083CF70F801C0834E
:10616000FF91EF91CF91BF91AF919F918F917F91CF
:106170006F915F914F913F912F911F910F91FF90E0
:10618000EF900F900FBE0F901F901895AA1BBB1B8E
:1061900051E107C0AA1FBB1FA617B70710F0A61B27
:1061A000B70B881F991F5A95A9F780959095BC0148
:1061B000CD01089597FB072E16F4009406D077FDC5
:1061C00008D0E4DF07FC05D03EF4909581959F4F01
:1061D0000895709561957F4F0895EE0FFF1F05900C
:1061E000F491E02D0994082E817006940694811D87
:1061F0000694811D0694811D0694811D0694811DBF
:106200000694801D08956927962769277827872790
:10621000782708952F923F924F925F926F927F92CC
:106220008F929F92AF92BF92CF92DF92EF92FF92A6
:106230000F931F93CF93DF93CDB7DEB7CA1BDB0B52
:106240000FB6F894DEBF0FBECDBF09942A883988F7
:1062500048885F846E847D848C849B84AA84B984FE
:10626000C884DF80EE80FD800C811B81AA81B9810A
:10627000CE0FD11D0FB6F894DEBF0FBECDBFED011E
:106280000895FB01DC0102C005900D924150504081
:10629000D8F70895FB01DC0104C08D9101908019AD
:1062A00021F441505040C8F7881B990B0895FB0119
:1062B000DC0102C001900D9241505040D8F7089582
:1062C000DC0101C06D9341505040E0F70895DC01BE
:1062D000CB01FC01F999FECF06C0F2BDE1BDF89AF1
:1062E000319600B40D9241505040B8F70895F99995
:1062F000FECF92BD81BDF89A992780B50895A8E197
:10630000B0E042E050E0E5CFDC01A40FB51F415002
:10631000504040F0CB01840F951F2E9105D0415085
:106320005040D8F70895262FF999FECF92BD81BD30
:10633000F89A019700B4021639F01FBA20BD0FB6C3
:10634000F894FA9AF99A0FBE08950396272FECDF76
:10635000EADF252FE9DF242FE7CF0196272FE4DF9F
:10636000E2CFDC01CB0102C02D9105D0415050405D
:10637000D8F70895262FF999FECF1FBA92BD81BD97
:1063800020BD0FB6F894FA9AF99A0FBE01960895B7
:10639000F894FFCF7F0B840B860B8B0B9B0B9B0B17
:1063A0009B0B9B0B9B0B9B0B9B0B9B0B8D0B910BD5
:1063B000940B990BA90BAF0BB30B9E11C411CA110F
:1063C000C411CA111C123D12CA11431350137F1E6F
:1063D000E71E871E511E551E8B1E591E8F1E9B1EAB
:1063E000651EE01E691E9F1E6D1EA31EC81E711E27
:1063F000A71ECF1E771EAD1EB51E5D1E931E611E0D
:10640000971E7B1EB11EBF1ED81EDE1E4B1E831E96
:10641000EE1E2C1E301E221E281E341E381E3C1E50
:10642000A520A52015211521B721D421C120C120E7
:10643000D92149225A225A22832D9E2DA52DEC2B9B
:10644000EC2BD72DE82DFB2D3C2E412E692E7A2EDC
:106450008F2E922EDA2BDE2B0D2C192C242C2F2C88
:10646000D82BD82BD82BD82B6F2D322C352C382C61
:0A647000612C9B2C9E2CA02CD42C38
:10647A0028081E0AB00A2D0E430E480E4D0E240E91
:10648A00AF00015001140000010001016B8AF2D42F
:10649A0069874B4C004422B684016201AC008A022F
:1064AA00A302C302F7F6F532F4366667F1F0C63096
:1064BA00313337929190973435E200E900EA00B51A
:1064CA0000B600B700CD008301CC008A0192019486
:1064DA00012102230224022502260227022A02B3EC
:1064EA0000B4006F0070009F01CB019F02A002E27E
:1064FA0000E900EA00B500B600B700CD008301CC80
:10650A00008A019201940121022302240225022613
:10651A000227022A02B300B4006F0070009F01CB69
:06652A00019F02A0020027
:00000001FF
